:020000040000FA
:020000005A287C
:08000800831A0B28B600030E59
:10001000B800BA131028B700030EB9008312BA173C
:100020000A08BB008A0183120313061E4A28A30A8A
:1000300064302302031C1D28A301C30B4128643034
:10004000C300BC0A0319BD0A3D083F02031D2F2847
:100050003C083E02031D2F283A10BC01BD01C20B13
:1000600041283C30C200C40A0319C50A44084002B2
:10007000031D412845084102031D4128C401C50153
:10008000BA14BA184728240A2302031C49288612E6
:100090004A2886160B103B088A00BA1F552883167B
:1000A000390E8300B70E370E0900380E8300B60EE6
:1000B000360E09008316103086008701D130850086
:1000C00006309F0083123C30C2006430C3008601BA
:1000D000A401A301AF01B501BA01B001C401C5017A
:1000E0001E30C600BC01BD0188308B0000003A14F0
:1000F000C521CA21D32183168E309F00831241303F
:100100009F000630A500A50B83281F151F19862800
:1001100083161E088312A6001E08A70003302702BC
:10012000031C9A28E8302602031C9A280330A700F3
:10013000E730A6002708B4002608B300A020C9288D
:10014000640003101030A500A801A901A60DA70D99
:10015000A80DA90DA50BB62829080F39AA00280E4D
:100160000F39A90028080F39A800080064002830BA
:100170008400BE2029308400BE20A628033000075A
:10018000AC00AC19800030300007AC00AC1B800024
:100190000034B50A07303502031DE828B5010030E8
:1001A0002F020319D828C60BD828AF011E30C6006D
:1001B000051AE828BA1CE128AF01C401C501BA102C
:1001C000E228AF0A04302F020319AF011E30C60027
:1001D0002F088207FA28F628F228EE2886210D300B
:1001E000AB002E296E210E30AB002E293A1CFA28C6
:1001F0003A10AF012908A8002A08A9002808B10070
:100200002908B2000A30AB003A1C0D29A7012408C6
:10021000A600A0200C30AA002E2901302F020319BD
:1002200014290B30AA0016290C30AA00B001B00A1C
:10023000B10B17290030B202031924290A30B1008A
:10024000B20B17290A30B00701302F02031D2A29EB
:1002500064212E293A182E293008A4003A1C352989
:10026000351C35290F30AB00AA00BA1C3F290F30CE
:10027000AB000030AA000C30A9000C30A800AD0182
:100280003730A50028302D07840002308A0000088E
:1002900013228A01AE002E08870002308A00012A4C
:1002A0008A016430AE006400AE0B5329AD0A0430FD
:1002B00003112D026400031D4229AD01A50B422943
:1002C0000000003087007B2806303502031D08003F
:1002D0003008A400A0000030AE210800063035022E
:1002E000031D080000303402031D7B290030330257
:1002F000031D7B29B30A3308BE00A0000130AE21E4
:100300003408BF00A0000230AE21080006303502DC
:10031000031D080000303402031D9329003033020E
:10032000031D9329B30A3308C000A0000330AE2197
:100330003408C100A0000430AE21C401C50108008A
:10034000031783168C18A2298C130C158B135530A8
:100350008D00AA308D008C140C1108008312031735
:100360008D0083012008831203178C00A0218301D4
:10037000BB218B170800E630A1000A30A200640000
:10038000A10BBF29A20BBF2908000030DC212008E7
:10039000A40008000130DC212008BE000230DC216E
:1003A0002008BF0008000330DC212008C000043012
:1003B000DC212008C1000800031783128D0083167A
:0E03C0008C130C1483120C080313A000080009
:0E0402002D088207072A0A2A0D2A102A8611C1
:1004100006145029861506115029061586105029F4
:1004200086140610502982073F3406345B344F345B
:1004300066346D347D3407347F346F3473345C3408
:08044000713478341C340034DF
:02400E00713D02
:00000001FF
